 pvr2dtest

 Timestamp is 4be8cee1 (Tue May 11 12:28:33 2010)

 Preferred load address is 00010000

 Start         Length     Name                   Class
 0001:00000000 00000004H .CRT$XCA                CODE
 0001:00000004 00000004H .CRT$XCZ                CODE
 0001:00000008 00000004H .CRT$XIA                CODE
 0001:0000000c 00000004H .CRT$XIZ                CODE
 0001:00000010 00000004H .CRT$XPA                CODE
 0001:00000014 00000004H .CRT$XPZ                CODE
 0001:00000018 00000004H .CRT$XTA                CODE
 0001:0000001c 00000004H .CRT$XTZ                CODE
 0001:00000020 00003060H .rdata                  CODE
 0001:00003080 00000026H .rdata$debug            CODE
 0001:000030a8 000042a4H .text                   CODE
 0001:0000734c 00000020H .xdata                  CODE
 0001:0000736c 00000034H .xdata$x                CODE
 0001:000073a0 00000028H .idata$2                CODE
 0001:000073c8 00000014H .idata$3                CODE
 0001:000073dc 000000e0H .idata$4                CODE
 0001:000074bc 000001bcH .idata$6                CODE
 0001:00007678 00000000H .edata                  CODE
 0002:00000000 000000e0H .idata$5                DATA
 0002:000000e0 00000020H .data                   DATA
 0002:00000100 0000000cH .bss                    DATA
 0003:00000000 000002f0H .pdata                  DATA

  Address         Publics by Value              Rva+Base       Lib:Object

 0000:00000000       ___safe_se_handler_count   00000000     <absolute>
 0000:00000000       ___safe_se_handler_table   00000000     <absolute>
 0001:00000000       __xc_a                     00011000     corelib0:crt0init.obj
 0001:00000004       __xc_z                     00011004     corelib0:crt0init.obj
 0001:00000008       __xi_a                     00011008     corelib0:crt0init.obj
 0001:0000000c       __xi_z                     0001100c     corelib0:crt0init.obj
 0001:00000010       __xp_a                     00011010     corelib0:crt0init.obj
 0001:00000014       __xp_z                     00011014     corelib0:crt0init.obj
 0001:00000018       __xt_a                     00011018     corelib0:crt0init.obj
 0001:0000001c       __xt_z                     0001101c     corelib0:crt0init.obj
 0001:00000070       ??_C@_0BL@IKOIDLAP@Invalid?5selection?5?$CI?$CFi?1?$CFi?$CJ?6?$AA@ 00011070     main.obj
 0001:0000008c       ??_C@_0CH@IGKHNFBD@?6Choose?5a?5test?1operation?5?$CIby?5num@ 0001108c     main.obj
 0001:000000b4       ??_C@_02IKAHHCAI@?$CFi?$AA@ 000110b4     main.obj
 0001:000000b8       ??_C@_07FCMIJJOF@?$CFu?4?5?$CFs?6?$AA@ 000110b8     main.obj
 0001:000000c0       ??_C@_01EEMJAFIK@?6?$AA@   000110c0     main.obj
 0001:000000c4       ??_C@_0BA@DHNFCGII@Start?5all?5tests?$AA@ 000110c4     main.obj
 0001:000000d4       ??_C@_0N@OPFFLDIA@Toggle?5debug?$AA@ 000110d4     main.obj
 0001:000000e4       ??_C@_0P@KLGDDFJI@Fill?5copy?5test?$AA@ 000110e4     main.obj
 0001:000000f4       ??_C@_0BC@JMJPADAB@Pattern?5copy?5test?$AA@ 000110f4     main.obj
 0001:00000108       ??_C@_0BI@MECNPGFM@Invert?5destination?5test?$AA@ 00011108     main.obj
 0001:00000120       ??_C@_0BI@OLJCEOMM@16?5bit?5source?5copy?5test?$AA@ 00011120     main.obj
 0001:00000138       ??_C@_0CA@MBMONALL@24?5bit?5clipped?5source?5copy?5test?$AA@ 00011138     main.obj
 0001:00000158       ??_C@_0CI@HFPJBNP@16?5bit?5source?5copy?5test?5with?5col@ 00011158     main.obj
 0001:00000180       ??_C@_0BN@LGNFKJAP@Masked?5destination?5copy?5test?$AA@ 00011180     main.obj
 0001:000001a0       ??_C@_0BP@CJPBFBLD@16?5bit?5masked?5source?5copy?5test?$AA@ 000111a0     main.obj
 0001:000001c0       ??_C@_0BI@BCPHBMOF@32?5bit?5alpha?5blend?5test?$AA@ 000111c0     main.obj
 0001:000001d8       ??_C@_04LBABLPF@Exit?$AA@  000111d8     main.obj
 0001:000027bc       ??_7CTestEnv@@6B@          000137bc     ctestenv.obj
 0001:00002864       ??_C@_0DE@PBHKGFGF@CTestEnv?3?3ConstructL?3?5Couldn?8t?5c@ 00013864     ctestenv.obj
 0001:00002940       ??_C@_0DJ@KKIIDLAA@DrawCheckboardBackground?5failed?5@ 00013940     graphics_op.obj
 0001:0000297c       ??_C@_0DK@MBOJPDFG@DrawCheckboardBackground?5failed?5@ 0001397c     graphics_op.obj
 0001:000029b8       ??_C@_0CA@NNDGBJEG@?5GOP?5Wait?5for?5Tests?5Complete?5?5?5?$AA@ 000139b8     graphics_op.obj
 0001:000029d8       ??_C@_0CA@PBLMLCCO@?5?5?5?5?5?5?5?5?5?5?5?5?5FAILED?$CB?5?5?5?5?5?5?5?5?5?5?5?$AA@ 000139d8     graphics_op.obj
 0001:000029f8       ??_C@_0CA@MDIFNAKF@?$CK?$CK?$CK?$CK?$CK?$CK?$CK?$CK?$CK?$CK?$CK?$CK?$CK?$CK?$CK?$CK?$CK?$CK?$CK?$CK?$CK?$CK?$CK?$CK?$CK?$CK?$CK?$CK?$CK?$CK?$CK?$AA@ 000139f8     graphics_op.obj
 0001:00002a18       ??_C@_0BL@ECFICAOA@?$DOGop?3?3WaitForTestsComplete?$AA@ 00013a18     graphics_op.obj
 0001:00002a34       ??_C@_0BF@BIHCPAAC@?$DOCGraphOp?3?3?$HOCGraphOp?$AA@ 00013a34     graphics_op.obj
 0001:00002a4c       ??_C@_0BE@BMGOGMEP@?$DOCGraphOp?3?3CGraphOp?$AA@ 00013a4c     graphics_op.obj
 0001:00002aac       ??_C@_0CA@PFFCLFAO@?5?5?5?5?5?5?5?5?5?5?5?5GOP?5Test?5?5?5?5?5?5?5?5?5?5?5?$AA@ 00013aac     graphics_op.obj
 0001:00002acc       ??_C@_0BP@HDNJMKLF@TGopBitBltAlphaChannel?5?$CI32bpp?$CJ?$AA@ 00013acc     graphics_op.obj
 0001:00002aec       ??_C@_0CC@DKEFJMNA@Blend?5complete?5bitmap?5with?5scree@ 00013aec     graphics_op.obj
 0001:00002b10       ??_C@_0CA@ONJNMDEO@TGopBitBlt?5?$CIsection?5from?524bpp?$CJ?$AA@ 00013b10     graphics_op.obj
 0001:00002b30       ??_C@_0CB@JBMIGPHB@Copy?5section?5of?5bitmap?5to?5screen@ 00013b30     graphics_op.obj
 0001:00002b54       ??_C@_0CA@BMHDGNMD@TGopBitBltMasked?5?$CISource?516bpp?$CJ?$AA@ 00013b54     graphics_op.obj
 0001:00002b74       ??_C@_0CI@DCAEAIEA@Copy?5complete?5bitmap?5referencing@ 00013b74     graphics_op.obj
 0001:00002b9c       ??_C@_0BI@CHDHNGPL@TGopBitBltMasked?5?$CIDest?$CJ?$AA@ 00013b9c     graphics_op.obj
 0001:00002bb4       ??_C@_0CH@LEPOLAEF@Copy?5screen?5section?5referencing?5@ 00013bb4     graphics_op.obj
 0001:00002bdc       ??_C@_0P@NIEAHFAK@TGopInvertRect?$AA@ 00013bdc     graphics_op.obj
 0001:00002bec       ??_C@_0CA@KGPGNCME@Inverts?5a?5section?5of?5the?5screen?$AA@ 00013bec     graphics_op.obj
 0001:00002c0c       ??_C@_0BK@MCACOCCA@TGopFilledRectWithPattern?$AA@ 00013c0c     graphics_op.obj
 0001:00002c28       ??_C@_0BN@IGGGBDFF@Copy?5small?5bitmap?5repeatedly?$AA@ 00013c28     graphics_op.obj
 0001:00002c48       ??_C@_0BJ@IMHEMMDF@TGopTransparency?5?$CI16bpp?$CJ?$AA@ 00013c48     graphics_op.obj
 0001:00002c64       ??_C@_0DG@MIKEPALE@Copy?5complete?5bitmap?5ignoring?5pi@ 00013c64     graphics_op.obj
 0001:00002c9c       ??_C@_0BD@MNHCHGP@TGopBitBlt?5?$CI16bpp?$CJ?$AA@ 00013c9c     graphics_op.obj
 0001:00002cb0       ??_C@_0CM@HHCMNDPA@TGopFilledRect?5?$CI16bpp?$CJ?5?$CL?54?5clipp@ 00013cb0     graphics_op.obj
 0001:00002cdc       ??_C@_0N@EGPBAMCG@?$DOGop?3?3DoTest?$AA@ 00013cdc     graphics_op.obj
 0001:000030b0       main                       000140b0 f   main.obj
 0001:00003254       WinMain                    00014254 f   main.obj
 0001:0000325c       ?ContextOpen@PVRIF_State@@AAAPAXXZ 0001425c f i ctestenv.obj
 0001:00003298       ??1PVRIF_State@@QAA@XZ     00014298 f i ctestenv.obj
 0001:000032b4       ?AccelInfo@CTestBitmap@@QAA?AVTAcceleratedBitmapInfo@@XZ 000142b4 f i ctestenv.obj
 0001:000032d4       ?ConstructL@CTestBitmap@@AAAXVTSize@@W4TDisplayMode@@@Z 000142d4 f   ctestenv.obj
 0001:00003350       ?ScreenAccelSpec@CTestEnv@@QAAPAU_PVR2DIFBitmapData_@@XZ 00014350 f   ctestenv.obj
 0001:0000335c       ?CopyData@CTestEnv@@AAAXPAE0JAAVTSize@@J@Z 0001435c f   ctestenv.obj
 0001:00003400       ?CopyImageData16bitSmall@CTestEnv@@AAAXAAVTAcceleratedBitmapInfo@@@Z 00014400 f   ctestenv.obj
 0001:00003444       ?CopyImageMaskData@CTestEnv@@AAAXAAVTAcceleratedBitmapInfo@@@Z 00014444 f   ctestenv.obj
 0001:00003488       ?CopyImageData@CTestEnv@@AAAXAAVTAcceleratedBitmapInfo@@@Z 00014488 f   ctestenv.obj
 0001:000035ac       ??1CTestEnv@@UAA@XZ        000145ac f   ctestenv.obj
 0001:000036dc       ??_ECTestEnv@@UAAPAXI@Z    000146dc f i ctestenv.obj
 0001:000036dc       ??_GCTestEnv@@UAAPAXI@Z    000146dc f i ctestenv.obj
 0001:00003708       ?NewL@CTestBitmap@@SAPAV1@PAVPVRIF_State@@VTSize@@W4TDisplayMode@@@Z 00014708 f   ctestenv.obj
 0001:000037a0       ?ConstructL@CTestEnv@@AAAXXZ 000147a0 f   ctestenv.obj
 0001:00003994       ?NewL@CTestEnv@@SAPAV1@XZ  00014994 f   ctestenv.obj
 0001:00003a2c       ??HTPoint@@QBA?AV0@ABV0@@Z 00014a2c f i graphics_op.obj
 0001:00003a68       ??HTPoint@@QBA?AV0@ABVTSize@@@Z 00014a68 f i graphics_op.obj
 0001:00003aa4       ??0TRect@@QAA@XZ           00014aa4 f i graphics_op.obj
 0001:00003ac0       ??1TRect@@QAA@XZ           00014ac0 f i graphics_op.obj
 0001:00003ac4       ?SetRect@TRect@@QAAXVTPoint@@VTSize@@@Z 00014ac4 f i graphics_op.obj
 0001:00003b10       ?Verbose1@CTestBase@@IAAXPBDZZ 00014b10 f i graphics_op.obj
 0001:00003b34       ?Size@CTestBitmap@@QBA?AVTSize@@XZ 00014b34 f i graphics_op.obj
 0001:00003b50       ?ScreenSize@CTestEnv@@QBA?AVTSize@@XZ 00014b50 f i graphics_op.obj
 0001:00003b6c       ?DrawCheckboardBackground@CGraphOp@@AAAXXZ 00014b6c f   graphics_op.obj
 0001:00003ec0       ?GetTestArea@CGraphOp@@AAA?AVTRect@@J@Z 00014ec0 f   graphics_op.obj
 0001:00003f68       ?WaitForTestsComplete@CGraphOp@@QAAJXZ 00014f68 f   graphics_op.obj
 0001:00003fd8       ??1CGraphOp@@QAA@XZ        00014fd8 f   graphics_op.obj
 0001:00003fe4       ??0CGraphOp@@QAA@PAVCTestEnv@@@Z 00014fe4 f   graphics_op.obj
 0001:00004008       ??0TGopBitBltTransparent@@QAA@ABVTPoint@@PAU_PVR2DIFBitmapData_@@ABVTRect@@ABVTGopTransparency@@@Z 00015008 f i graphics_op.obj
 0001:0000408c       ?DoTest@CGraphOp@@QAAJJ_N@Z 0001508c f   graphics_op.obj
 0001:00004774       ?VPrint@CTestBase@@AAAXW4VERBOSE_LEVEL_tag@1@PBDPAD@Z 00015774 f   testbase.obj
 0001:000047b8       ?Error@CTestBase@@IAAXPBDZZ 000157b8 f   testbase.obj
 0001:00004808       ?ConstructL@CPVR2DAppView@@QAAXXZ 00015808 f   PVR2DTest.obj
 0001:0000488c       ?DrawAllTestsNow@CPVR2DAppView@@QAAXXZ 0001588c f   PVR2DTest.obj
 0001:000048c4       ??1CPVR2DAppView@@QAA@XZ   000158c4 f   PVR2DTest.obj
 0001:00004908       ??1CPVR2DAppUi@@QAA@XZ     00015908 f   PVR2DTest.obj
 0001:0000492c       ?HandleCommandL@CPVR2DAppUi@@QAAXJ@Z 0001592c f   PVR2DTest.obj
 0001:00004a54       ?NewL@CPVR2DAppView@@SAPAV1@XZ 00015a54 f   PVR2DTest.obj
 0001:00004ac8       ?ConstructL@CPVR2DAppUi@@QAAXXZ 00015ac8 f   PVR2DTest.obj
 0001:00004adc       ?ConstructL@CPVR2DHardwareGraphicsAccelerator@@IAAXXZ 00015adc f   pvr2dif_accelhard.obj
 0001:00004b14       ?Operation@CPVR2DHardwareGraphicsAccelerator@@QAAJABVTGraphicsOperation@@JPAVTRect@@@Z 00015b14 f   pvr2dif_accelhard.obj
 0001:00004b40       ?QueryOpsComplete@CPVR2DHardwareGraphicsAccelerator@@QAAJW4eQueryOpsMode@1@@Z 00015b40 f   pvr2dif_accelhard.obj
 0001:00004b5c       ??1CPVR2DHardwareGraphicsAccelerator@@QAA@XZ 00015b5c f   pvr2dif_accelhard.obj
 0001:00004bb8       ?NewL@CPVR2DHardwareGraphicsAccelerator@@SAPAV1@PAVPVRIF_State@@PAU_PVR2DIFBitmapData_@@@Z 00015bb8 f   pvr2dif_accelhard.obj
 0001:00004c3c       ?Operation@CPVR2DHardwareGraphicsAccelerator@@QAAJABVTGraphicsOperation@@@Z 00015c3c f   pvr2dif_accelhard.obj
 0001:00004c68       ?PVR2DIF_HardwareBitmapGetInfo@@YAJPAU_PVR2DIFBitmapData_@@AAVTAcceleratedBitmapInfo@@@Z 00015c68 f   pvr2dif_bitmap.obj
 0001:00004db4       ?PVR2DIF_HardwareBitmapScreenReference@@YAJPAU_PVR2DIFBitmapData_@@PAVPVRIF_State@@@Z 00015db4 f   pvr2dif_bitmap.obj
 0001:00004e50       ?PVR2DIF_HardwareBitmapCreate@@YAJPAU_PVR2DIFBitmapData_@@PAVPVRIF_State@@W4TDisplayMode@@VTSize@@@Z 00015e50 f   pvr2dif_bitmap.obj
 0001:00004f50       ?PVR2DIF_HardwareBitmapDestroy@@YAXPAU_PVR2DIFBitmapData_@@PAVPVRIF_State@@@Z 00015f50 f   pvr2dif_bitmap.obj
 0001:00004f60       ?Size@TRect@@QBA?AVTSize@@XZ 00015f60 f i pvr2dif_ops.obj
 0001:00004f8c       ?Color@TGopTransparency@@QBA?AVTRgb@@XZ 00015f8c f i pvr2dif_ops.obj
 0001:00005118       ?OpQueryGraphicsOpsComplete@@YAJPAVPVRIF_State@@PAU_PVR2DIFBitmapData_@@_N@Z 00016118 f   pvr2dif_ops.obj
 0001:00005314       ?OpGraphicsOperation@@YAJPAVPVRIF_State@@PAU_PVR2DIFBitmapData_@@ABVTGraphicsOperation@@JPAVTRect@@@Z 00016314 f   pvr2dif_ops.obj
 0001:00005834       ?ContextConnect@PVRIF_State@@AAAPAXXZ 00016834 f   pvr2dif_state.obj
 0001:000058b8       PVR2DEnumerateDevices      000168b8 f   libpvr2d:pvr2dinit.obj
 0001:00005c88       PVR2DCreateDeviceContext   00016c88 f   libpvr2d:pvr2dinit.obj
 0001:00005eb0       PVR2DDestroyDeviceContext  00016eb0 f   libpvr2d:pvr2dinit.obj
 0001:00005fb4       PVR2DGetFrameBuffer        00016fb4 f   libpvr2d:pvr2dmode.obj
 0001:00005ff0       PVR2DGetScreenMode         00016ff0 f   libpvr2d:pvr2dmode.obj
 0001:000060cc       PVR2DMemAlloc              000170cc f   libpvr2d:pvr2dmem.obj
 0001:00006188       PVR2DMemFree               00017188 f   libpvr2d:pvr2dmem.obj
 0001:0000624c       GetPvrSrvPixelFormat       0001724c f   libpvr2d:pvr2dblt.obj
 0001:000062bc       PVR2DQueryBlitsComplete    000172bc f   libpvr2d:pvr2dblt.obj
 0001:00006bd8       PVR2DBltClipped            00017bd8 f   libpvr2d:pvr2dblt.obj
 0001:00006bdc       DestroyFlipChain           00017bdc f   libpvr2d:pvr2dflip.obj
 0001:00006cac       PVRSRVDisconnect           00017cac f   srvclum:SRVCLUM.dll
 0001:00006cbc       PVRSRVCloseDCDevice        00017cbc f   srvclum:SRVCLUM.dll
 0001:00006ccc       PVRSRVMemCopy              00017ccc f   srvclum:SRVCLUM.dll
 0001:00006cdc       PVRSRVGetDCInfo            00017cdc f   srvclum:SRVCLUM.dll
 0001:00006cec       PVRSRVOpenDCDevice         00017cec f   srvclum:SRVCLUM.dll
 0001:00006cfc       PVRSRVFreeUserModeMem      00017cfc f   srvclum:SRVCLUM.dll
 0001:00006d0c       PVRSRVCallocUserModeMem    00017d0c f   srvclum:SRVCLUM.dll
 0001:00006d1c       PVRSRVAcquireDeviceData    00017d1c f   srvclum:SRVCLUM.dll
 0001:00006d2c       PVRSRVEnumerateDevices     00017d2c f   srvclum:SRVCLUM.dll
 0001:00006d3c       PVRSRVEnumerateDeviceClass 00017d3c f   srvclum:SRVCLUM.dll
 0001:00006d4c       PVRSRVConnect              00017d4c f   srvclum:SRVCLUM.dll
 0001:00006d5c       PVRSRVUnmapDeviceClassMemory 00017d5c f   srvclum:SRVCLUM.dll
 0001:00006d6c       PVRSRVMapDeviceClassMemory 00017d6c f   srvclum:SRVCLUM.dll
 0001:00006d7c       PVRSRVGetDCSystemBuffer    00017d7c f   srvclum:SRVCLUM.dll
 0001:00006d8c       PVRSRVEnumDCDims           00017d8c f   srvclum:SRVCLUM.dll
 0001:00006d9c       PVRSRVAllocUserModeMem     00017d9c f   srvclum:SRVCLUM.dll
 0001:00006dac       PVRSRVEnumDCFormats        00017dac f   srvclum:SRVCLUM.dll
 0001:00006dbc       PVRSRVDestroyDeviceMemContext 00017dbc f   srvclum:SRVCLUM.dll
 0001:00006dcc       PVRSRVReleaseMiscInfo      00017dcc f   srvclum:SRVCLUM.dll
 0001:00006ddc       SGXDestroyTransferContext  00017ddc f   srvclum:SRVCLUM.dll
 0001:00006dec       SGXCreateTransferContext   00017dec f   srvclum:SRVCLUM.dll
 0001:00006dfc       PVRSRVCreateDeviceMemContext 00017dfc f   srvclum:SRVCLUM.dll
 0001:00006e0c       PVRSRVGetMiscInfo          00017e0c f   srvclum:SRVCLUM.dll
 0001:00006e1c       PVRSRVAllocDeviceMem       00017e1c f   srvclum:SRVCLUM.dll
 0001:00006e2c       PVRSRVMemSet               00017e2c f   srvclum:SRVCLUM.dll
 0001:00006e3c       PVRSRVFreeDeviceMem        00017e3c f   srvclum:SRVCLUM.dll
 0001:00006e4c       PVRSRVUnwrapExtMemory      00017e4c f   srvclum:SRVCLUM.dll
 0001:00006e5c       PVRSRVUnmapDeviceMemory    00017e5c f   srvclum:SRVCLUM.dll
 0001:00006e6c       PVRSRVEventObjectWait      00017e6c f   srvclum:SRVCLUM.dll
 0001:00006e7c       SGX2DQueryBlitsComplete    00017e7c f   srvclum:SRVCLUM.dll
 0001:00006e8c       PVRSRVClockus              00017e8c f   srvclum:SRVCLUM.dll
 0001:00006e9c       SGXQueueTransfer           00017e9c f   srvclum:SRVCLUM.dll
 0001:00006eac       PVRSRVDestroyDCSwapChain   00017eac f   srvclum:SRVCLUM.dll
 0001:00006ebc       PVRSRVSwapToDCSystem       00017ebc f   srvclum:SRVCLUM.dll
 0001:00006f4c       WinMainCRTStartup          00017f4c f   corelib0:pegwmain.obj
 0001:00006f80       __GSHandlerCheckCommon     00017f80 f   corelib0:gshandler.obj
 0001:00006fbc       __GSHandlerCheck           00017fbc f   corelib0:gshandler.obj
 0001:00006fe0       __security_init_cookie     00017fe0 f   corelib0:seccinit.obj
 0001:0000703c       __security_check_cookie    0001803c f   corelib0:armsecgs.obj
 0001:00007050       __gsfailure                00018050 f   corelib0:armsecgs.obj
 0001:0000715c       exit                       0001815c f   corelib0:cexit.obj
 0001:00007174       _exit                      00018174 f   corelib0:cexit.obj
 0001:000071b4       _initterm                  000181b4 f   corelib0:crt0dat.obj
 0001:000071e8       _cinit                     000181e8 f   corelib0:crt0dat.obj
 0001:0000721c       scanf                      0001821c f   corelib1:COREDLL.dll
 0001:0000722c       printf                     0001822c f   corelib1:COREDLL.dll
 0001:0000723c       __CxxFrameHandler3         0001823c f   corelib1:COREDLL.dll
 0001:0000724c       memcpy                     0001824c f   corelib1:COREDLL.dll
 0001:0000725c       __CxxThrowException        0001825c f   corelib1:COREDLL.dll
 0001:0000726c       ??_7type_info@@6B@         0001826c f   corelib1:COREDLL.dll
 0001:0000727c       ??3@YAXPAX@Z               0001827c f   corelib1:COREDLL.dll
 0001:0000728c       ??2@YAPAXI@Z               0001828c f   corelib1:COREDLL.dll
 0001:0000729c       ??_M@YAXPAXIHP6AX0@Z@Z     0001829c f   corelib1:COREDLL.dll
 0001:000072ac       ??_L@YAXPAXIHP6AX0@Z1@Z    000182ac f   corelib1:COREDLL.dll
 0001:000072bc       _vsnprintf                 000182bc f   corelib1:COREDLL.dll
 0001:000072cc       memset                     000182cc f   corelib1:COREDLL.dll
 0001:000072dc       free                       000182dc f   corelib1:COREDLL.dll
 0001:000072ec       malloc                     000182ec f   corelib1:COREDLL.dll
 0001:000072fc       _XcptFilter                000182fc f   corelib1:COREDLL.dll
 0001:0000730c       __C_specific_handler       0001830c f   corelib1:COREDLL.dll
 0001:0000731c       __security_gen_cookie2     0001831c f   corelib1:COREDLL.dll
 0001:0000732c       __report_gsfailure         0001832c f   corelib1:COREDLL.dll
 0001:0000733c       TerminateProcess           0001833c f   coredll:COREDLL.dll
 0001:0000736c       _TI1?AVXError@@            0001836c     ctestenv.obj
 0001:0000737c       _CTA1?AVXError@@           0001837c     ctestenv.obj
 0001:00007384       _CT??_R0?AVXError@@@84     00018384     ctestenv.obj
 0001:000073a0       __IMPORT_DESCRIPTOR_SRVCLUM 000183a0     srvclum:SRVCLUM.dll
 0001:000073b4       __IMPORT_DESCRIPTOR_COREDLL 000183b4     corelib1:COREDLL.dll
 0001:000073c8       __NULL_IMPORT_DESCRIPTOR   000183c8     srvclum:SRVCLUM.dll
 0002:00000000       __imp_TerminateProcess     00019000     coredll:COREDLL.dll
 0002:00000004       __imp___report_gsfailure   00019004     corelib1:COREDLL.dll
 0002:00000008       __imp___security_gen_cookie2 00019008     corelib1:COREDLL.dll
 0002:0000000c       __imp___C_specific_handler 0001900c     corelib1:COREDLL.dll
 0002:00000010       __imp__XcptFilter          00019010     corelib1:COREDLL.dll
 0002:00000014       __imp_malloc               00019014     corelib1:COREDLL.dll
 0002:00000018       __imp_free                 00019018     corelib1:COREDLL.dll
 0002:0000001c       __imp_memset               0001901c     corelib1:COREDLL.dll
 0002:00000020       __imp__vsnprintf           00019020     corelib1:COREDLL.dll
 0002:00000024       __imp___rt_sdiv            00019024     corelib1:COREDLL.dll
 0002:00000028       __imp_??_L@YAXPAXIHP6AX0@Z1@Z 00019028     corelib1:COREDLL.dll
 0002:0000002c       __imp_??_M@YAXPAXIHP6AX0@Z@Z 0001902c     corelib1:COREDLL.dll
 0002:00000030       __imp_??2@YAPAXI@Z         00019030     corelib1:COREDLL.dll
 0002:00000034       __imp_??3@YAXPAX@Z         00019034     corelib1:COREDLL.dll
 0002:00000038       __imp_??_7type_info@@6B@   00019038     corelib1:COREDLL.dll
 0002:0000003c       __imp___CxxThrowException  0001903c     corelib1:COREDLL.dll
 0002:00000040       __imp_memcpy               00019040     corelib1:COREDLL.dll
 0002:00000044       __imp___CxxFrameHandler3   00019044     corelib1:COREDLL.dll
 0002:00000048       __imp_printf               00019048     corelib1:COREDLL.dll
 0002:0000004c       __imp_scanf                0001904c     corelib1:COREDLL.dll
 0002:00000050       \177COREDLL_NULL_THUNK_DATA 00019050     corelib1:COREDLL.dll
 0002:00000054       __imp_PVRSRVAllocDeviceMem 00019054     srvclum:SRVCLUM.dll
 0002:00000058       __imp_PVRSRVMemSet         00019058     srvclum:SRVCLUM.dll
 0002:0000005c       __imp_PVRSRVFreeDeviceMem  0001905c     srvclum:SRVCLUM.dll
 0002:00000060       __imp_PVRSRVUnwrapExtMemory 00019060     srvclum:SRVCLUM.dll
 0002:00000064       __imp_PVRSRVUnmapDeviceMemory 00019064     srvclum:SRVCLUM.dll
 0002:00000068       __imp_PVRSRVEventObjectWait 00019068     srvclum:SRVCLUM.dll
 0002:0000006c       __imp_PVRSRVGetMiscInfo    0001906c     srvclum:SRVCLUM.dll
 0002:00000070       __imp_PVRSRVClockus        00019070     srvclum:SRVCLUM.dll
 0002:00000074       __imp_SGXQueueTransfer     00019074     srvclum:SRVCLUM.dll
 0002:00000078       __imp_PVRSRVDestroyDCSwapChain 00019078     srvclum:SRVCLUM.dll
 0002:0000007c       __imp_PVRSRVSwapToDCSystem 0001907c     srvclum:SRVCLUM.dll
 0002:00000080       __imp_PVRSRVCreateDeviceMemContext 00019080     srvclum:SRVCLUM.dll
 0002:00000084       __imp_SGXCreateTransferContext 00019084     srvclum:SRVCLUM.dll
 0002:00000088       __imp_SGXDestroyTransferContext 00019088     srvclum:SRVCLUM.dll
 0002:0000008c       __imp_PVRSRVReleaseMiscInfo 0001908c     srvclum:SRVCLUM.dll
 0002:00000090       __imp_PVRSRVDestroyDeviceMemContext 00019090     srvclum:SRVCLUM.dll
 0002:00000094       __imp_PVRSRVEnumDCFormats  00019094     srvclum:SRVCLUM.dll
 0002:00000098       __imp_PVRSRVAllocUserModeMem 00019098     srvclum:SRVCLUM.dll
 0002:0000009c       __imp_PVRSRVEnumDCDims     0001909c     srvclum:SRVCLUM.dll
 0002:000000a0       __imp_PVRSRVGetDCSystemBuffer 000190a0     srvclum:SRVCLUM.dll
 0002:000000a4       __imp_PVRSRVMapDeviceClassMemory 000190a4     srvclum:SRVCLUM.dll
 0002:000000a8       __imp_PVRSRVUnmapDeviceClassMemory 000190a8     srvclum:SRVCLUM.dll
 0002:000000ac       __imp_PVRSRVConnect        000190ac     srvclum:SRVCLUM.dll
 0002:000000b0       __imp_PVRSRVEnumerateDeviceClass 000190b0     srvclum:SRVCLUM.dll
 0002:000000b4       __imp_PVRSRVEnumerateDevices 000190b4     srvclum:SRVCLUM.dll
 0002:000000b8       __imp_PVRSRVAcquireDeviceData 000190b8     srvclum:SRVCLUM.dll
 0002:000000bc       __imp_PVRSRVCallocUserModeMem 000190bc     srvclum:SRVCLUM.dll
 0002:000000c0       __imp_PVRSRVFreeUserModeMem 000190c0     srvclum:SRVCLUM.dll
 0002:000000c4       __imp_PVRSRVOpenDCDevice   000190c4     srvclum:SRVCLUM.dll
 0002:000000c8       __imp_PVRSRVGetDCInfo      000190c8     srvclum:SRVCLUM.dll
 0002:000000cc       __imp_PVRSRVMemCopy        000190cc     srvclum:SRVCLUM.dll
 0002:000000d0       __imp_PVRSRVCloseDCDevice  000190d0     srvclum:SRVCLUM.dll
 0002:000000d4       __imp_SGX2DQueryBlitsComplete 000190d4     srvclum:SRVCLUM.dll
 0002:000000d8       __imp_PVRSRVDisconnect     000190d8     srvclum:SRVCLUM.dll
 0002:000000dc       \177SRVCLUM_NULL_THUNK_DATA 000190dc     srvclum:SRVCLUM.dll
 0002:000000e0       ??_R0?AVXError@@@8         000190e0     ctestenv.obj
 0002:000000f8       __security_cookie          000190f8     corelib0:seccinit.obj
 0002:000000fc       __security_cookie_complement 000190fc     corelib0:seccinit.obj
 0002:00000100       _exitflag                  00019100     corelib0:cexit.obj
 0002:00000104       __onexitend                00019104     <common>
 0002:00000108       __onexitbegin              00019108     <common>

 entry point at        0001:00006f4c

 Static symbols

 0001:00003200       __unwind$34663             00014200 f   main.obj
 0001:000036bc       __unwind$35162             000146bc f   ctestenv.obj
 0001:00003764       __catch$35363              00014764 f   ctestenv.obj
 0001:000039ec       __catch$35562              000149ec f   ctestenv.obj
 0001:00003e8c       __unwind$35861             00014e8c f   graphics_op.obj
 0001:000046f0       __unwind$36479             000156f0 f   graphics_op.obj
 0001:0000485c       __catch$34762              0001585c f   PVR2DTest.obj
 0001:00004878       __unwind$34763             00015878 f   PVR2DTest.obj
 0001:00004a8c       __catch$35064              00015a8c f   PVR2DTest.obj
 0001:00004d18       ?GlobalDataInit@@YAJPAU_PVR2DIFBitmapData_@@W4PVR2DFORMAT@@IIKPAU_PVR2DMEMINFO@@@Z 00015d18 f   pvr2dif_bitmap.obj
 0001:00004fb8       ?_ConvertColour@@YAJAAKW4PVR2DFORMAT@@VTRgb@@@Z 00015fb8 f   pvr2dif_ops.obj
 0001:00005030       ?_DoPVR2DBlit@@YAJPAXPAU_PVR2DBLTINFO@@JPAVTRect@@PAU_PVR2DIFBitmapData_@@@Z 00016030 f   pvr2dif_ops.obj
 0001:00005148       ?PVR2DIF_InitBlitInfo@@YAXAAU_PVR2DBLTINFO@@PBU_PVR2DIFBitmapData_@@1ABVTRect@@2@Z 00016148 f   pvr2dif_ops.obj
 0001:00005208       ?DoFilledRectUsingDrawMode@@YAJAAU_PVR2DBLTINFO@@PBU_PVR2DIFBitmapData_@@ABVTGopFilledRectUsingDrawMode@@@Z 00016208 f   pvr2dif_ops.obj
 0001:00005aa0       InitDisplayDevice          00016aa0 f   libpvr2d:pvr2dinit.obj
 0001:00006398       AltBltClipped              00017398 f   libpvr2d:pvr2dblt.obj
 0001:00006ed4       WinMainCRTStartupHelper    00017ed4 f   corelib0:pegwmain.obj
 0001:00007094       doexit                     00018094 f   corelib0:cexit.obj
